:1000000010C017C016C015C014C013C012C011C054
:1000100010C00FC00EC00DC00CC00BC00AC009C07C
:1000200008C011241FBECFE5D1E0DEBFCDBF6ED02A
:100030008EC0E6CF80E88BBB2FEF34E39CE02150ED
:1000400030409040E1F700C000001BBA2FEF34E3CE
:100050009CE0215030409040E1F700C000008BBB95
:100060002FEF34E39CE0215030409040E1F700C096
:1000700000001BBA2FEF34E39CE021503040904049
:10008000E1F700C000008BBB2FEF34E38CE0215080
:1000900030408040E1F700C000001BBA089580E8BE
:1000A0008BBB2FE734E89EE1215030409040E1F7D0
:1000B00000C000001BBA2FE734E89EE12150304019
:1000C0009040E1F700C000008BBB2FE734E88EE1E1
:1000D000215030408040E1F700C000001BBA089575
:1000E00080E88BBB2FE784E89EE121508040904060
:1000F000E1F700C000001BBA2FE784E89EE1215021
:1001000080409040E1F700C00000089587EF8ABB6F
:1001100017BACB9BFECF2FE784E89EE121508040A9
:100120009040E1F700C00000CB9B02C083DFF1CF1D
:100130002FE382E49FE0215080409040E1F700C02F
:100140000000CB9B02C0ABDFE4CFCADFE2CFF89464
:02015000FFCFDF
:00000001FF
